:08000000F017002005290000A3
:100400000000000000000000FFFFFFFFBE08FFFF2C
:1004100008B50B4802F03EFDC023F822DB011202B2
:100420001978FF2904D101339342F9D1002005E066
:10043000044A00209A4240414042184008BDC0464C
:1004400008430000FFF70000031C3038C0B200B5BD
:10045000092807D9181C3738C0B20F2802D9181C30
:100460005738C0B200BD0000F8B50C4D0C4F0D4E12
:100470002868391C326802F09BF9041E04D00A482F
:1004800002F008FD012407E08022381CFF21D20081
:1004900002F0EAFB34602C60201CF8BDF4FDFF1F65
:1004A000ECF8FF1FF8FDFF1F1C430000F7B5CB065B
:1004B00002D52023137001324BB2002B04DA302313
:1004C000137078235370023220230B4000930823CB
:1004D0000B404026019307230E4019400F1C0429AE
:1004E00000D90427FFB27F000F21141C3B1C8C464F
:1004F000013BDBB2FF2B15D09D00011CE9400D1C18
:1005000061460D40291C3031392908D9009900294C
:1005100002D0291C373102E0291C5731C9B22170A1
:100520000134E5E7019BD019002B04D00D230370A3
:100530000A2343700230002E00D10670FEBD1FB5A5
:100540006A46FFF7B3FF684602F0A4FC05B000BDA1
:1005500008B5144802F09EFC134802F09BFC1348B7
:1005600002F098FCC1208421C001FFF7E8FF104889
:1005700002F090FC84210F48FFF7E1FF0E4802F0E3
:1005800089FC0E4802F086FC0D4802F083FC0D4801
:1005900002F080FC0C4802F07DFC0C4802F07AFC72
:1005A00008BDC0463F4300005B43000075430000A8
:1005B00077430000FFF70000794300007D4300000F
:1005C0008F430000A2430000B5430000C743000072
:1005D000F0B5AA4DA5B02C68867B002C01D0A84CA4
:1005E00034E027210A2369440B706A4620231384D0
:1005F00040235384B4235B00262093846844612302
:100600000AA904700B70201C032108AA02F00CFB3D
:100610009C4F3870002803D00521221C02F052FAAA
:10062000994B3A781A70FFF793FFFF2104229748FD
:1006300002F01AFB80229648FF21D20002F014FB40
:1006400001232B60CBE7E778002F07D0301C211C5B
:10065000052202F04DFA0028F5D133E02379012B71
:1006600002D102F00FF9F1E7032B0AD1FFF7FCFEEC
:100670001023002800D1042386482B6002F00AFCD6
:10068000E4E701F0B5FA844B844A1F60844B1F688D
:100690003A401A60834B1868420052081A60824A36
:1006A00001235B421360814AC1201360804AC0016C
:1006B0001360804A1360804A1360804A136002F01E
:1006C000DDF9C3E72B68190600D580E27C4D6D4E3D
:1006D0002F683078E119012202F00AFA002800D1CF
:1006E00075E22F68E35D0A2BF0D0644E3268042A6D
:1006F00000D19CE005DC012A0BD0022A00D05EE28A
:100700006FE0202A6DD0402A6BD0102A00D14DE234
:1007100055E20D2B4CD100232B60022F44D12378BE
:1007200020229343442B08D163789343432B3BD13E
:10073000644802F0AFFB376041E24C2B08D163788C
:100740009343442B30D1604802F0A4FB042335E2EC
:10075000472B0BD16378202293434F2B24D15B4846
:1007600002F098FB61200421022224E24D2B09D1E2
:1007700063782025AB43452B16D1554802F08AFB00
:1007800035601CE2422B0FD1637820229343432B28
:100790000AD1FFF73DFE002801D14E4805E0942123
:1007A000FFF7CDFE4C4800E04C4802F073FB06E238
:1007B0003F2B04D100232B60FFF7CAFEFFE1314E2F
:1007C000E119307802F044FB2B68E15C5A1C2A6086
:1007D000082900D0F3E1013B012A00DC00232B6053
:1007E000EDE1237820218B43592B1CD18A4204D17F
:1007F0003B4802F04FFB4023E0E1402A02D101F0E8
:10080000BBFFDCE1374802F045FBC0209821C00166
:10081000090201F0B8FF471C03D0002810D132486C
:1008200002E0324800E0324802F034FB08E0032BDB
:1008300008D1304802F02EFB00232B60FFF788FE22
:100840000123BBE17A1C2A600D2B00D0B7E123788D
:1008500020218B43532B00D093E008AB1E7A00215C
:1008600006965E7A601CA2180596089F099E049061
:10087000039101910D1C079252E0C04600FEFF1F3C
:10088000F4FCFF1FDCF8FF1FDAF8FF1FECFCFF1F72
:10089000ECF8FF1FE243000010E000E0FFC3FBFFA5
:1008A000348004400070044080E100E084E100E016
:1008B00088E100E080E200E084E200E088E200E01D
:1008C000F0FCFF1FE5430000FE4300001E44000053
:1008D00038440000504400005C4400006C440000B8
:1008E00074440000A7440000BB440000CA44000058
:1008F000D7440000E7440000049B1878042D00DB77
:1009000087E0022D72DC002D3DDDFFF79DFD022307
:100910005D1B9D40A8400643049A029D013204924B
:10092000049B079883422CD26A1C02920A2DE3DDB5
:10093000C82D00DAD5E0C92D74DDCA2D00D0D0E075
:10094000059B29226A4413703A0C3B0E9B18DBB2BC
:10095000DB19DBB23A0A09969B18039EDBB29B199E
:100960000699DB43059E0AA8DBB2017008970320B5
:100970009E4200D0E5E0019EF50FAD196D10002DEF
:100980005EDC0120DDE0002D00D0AAE0302800D19F
:1009900005E1352800D102E1031C373BDBB2022B15
:1009A00000D9C7E008972922059F0AA96A44087060
:1009B00017700996FFF758FD002801D00020C0E00D
:1009C0000020011C021C01F0F3FEC120C00181497E
:1009D000042201F0EDFE0028F0D17F487F4B8360B8
:1009E00001F03AF80028E9D10620AAE0069AF1B20F
:1009F00003917600312A02D1063E082308E00699C9
:100A0000322903D10622083E029202E00A3E042364
:100A10000293FFF719FD02990B235B1A9B00984084
:100A2000074379E7049A1078FFF70EFDC9235D1B91
:100A3000AD00059BA840051C1D43EDB205956BE775
:100A4000674887421DD8674B9F4218D96B462A33A7
:100A5000604E0BE0644FB118C9191F780132013D97
:100A60000F7008920133002D00D198E0089A191CEC
:100A70008242EFD9089B5D48EA18824204D90420DB
:100A80005FE069462A31F5E753480668B24200D96B
:100A90000260574A574E1068574F002802D1136022
:100AA00033600CE03268934209D038689A1A121801
:100AB0003360524B3A60AA1802209A4241D83A68F1
:100AC0004F4880182A1C02F0D8F8386831682B1873
:100AD000CE224D193B603560920093425FD90520CC
:100AE0002FE0049A019B012110780B420FD0DD0FFB
:100AF000ED180D41FFF7A8FC08AA5519AB7A184369
:100B0000C0B2A872039BC018C0B2039009E0FFF7FF
:100B10009BFC019908AACB0F5B185B10D31800014E
:100B20009872019B01330193B34200DAF4E6C821C5
:100B30000291F1E6069001202E1C05952F1C0290D3
:100B4000EAE603F07DFB0D042A06191B0F002D4871
:100B500000E02D4802F09EF910222C4B1A6021E093
:100B60002B48F7E72B4802F095F901226120142168
:100B700002F04EFB0822F0E7274811E0274802F078
:100B800089F903226120042102F042FB244B002258
:100B90001A601E4B80221A6019E02248DAE72248C8
:100BA00002F078F91E4B00221A6008E0122B06D1E1
:100BB00061200421012202F02BFB08233360184B33
:100BC0001968FF2900DC81E500221A607EE525B066
:100BD000F0BDC046ECFCFF1FE0F8FF1FF34400002F
:100BE000836000007F600000809FFFFFFFF7000030
:100BF000F4FDFF1FFCFDFF1FF8FDFF1F9B0300001E
:100C0000ECF8FF1FFF4400002145000000FEFF1F1D
:100C1000414500006A450000884500008A45000003
:100C2000F0FCFF1F8D450000B9440000134B10B5C8
:100C30001A6801242240124B12D0C1200024C001A6
:100C40001C80036801330CD00E4B1B68013308D0A5
:100C5000C023DB011B68013303D001F00FFF00E06C
:100C60001A80FFF7D5FB002807D0002C05D1C02043
:100C70009821C001090201F086FD10BD50F00F401F
:100C8000FE1700208460000000B5021C8032C37A89
:100C9000202B03D090420CD02030F8E7C27F837F16
:100CA00012061B04D218437F1B02D218037FD018F0
:100CB00000E0012000BD000070B50D1C022A48D0E4
:100CC000042A02D0002A34D10AE003780324822BBC
:100CD00042D1224B224918780D2202F0B9F83BE0AC
:100CE000017880230A1C9A43212A34D1C37982795E
:100CF0001E021C4C164349B2268000292BDA41788B
:100D0000FE2902D0FF290FD025E08178002922D1C9
:100D1000C17800291FD1012A1DD1002B1BD1124BF4
:100D20001249187802F094F80024082D14D9083DCF
:100D3000ADB20C4B1A88181C002A02D10024048082
:100D40000AE00B4900240C709542F7D2551B1D8018
:100D500002E0002400E00424201C70BD30000020CC
:100D6000C0F8FF1FBC0800203100002040460000F2
:100D700020FEFF1F10B5184A031C1078441C147085
:100D8000141C032826D8154A03F05AFA020B181F20
:100D9000F02014880001084020430C03204309067A
:100DA00007E00C09F02020400C02204314880905BC
:100DB0002043090F1180188002330BE010880901CD
:100DC0000143002010801980F6E7C9B2002020708E
:100DD00011801980181C10BD3800002008FEFF1F6C
:100DE000F7B5A94D8026B600041C00216869321CA5
:100DF00001F03AFF2F1C002C5BD0022C00D98BE0B5
:100E00006C69EB2323709023A370A049E01C02F0CF
:100E100069F83F222E852276FF22A276F82262759B
:100E20009B493C2201260023022762700822E372BC
:100E30002674E37422752773A773A774201C0A70A5
:100E4000E3750423A675AB609249363001F015FFB7
:100E5000914B8F491E60AB68EE611A1C2032013B3A
:100E6000EA602B620B7880226373631DDA77E31DDF
:100E70002922DA779B19DE779B19DF7703229B19EA
:100E8000DA779B19261C04222B36DA7783490B224A
:100E9000301C01F0F2FE281C0B224930311C01F0FD
:100EA000ECFEFF2355225B00E2547D4BAA22E25464
:100EB000E7E06B69C0220221FF329954E0220C2145
:100EC00052009954E1220B2152009954C422382136
:100ED000FF329954E222F82152009954C622B821D7
:100EE000FF3299540121E3228A409954E522FF21DF
:100EF00052009954CC220721FF329954E622520025
:100F00009C54CE22FF329C54FF225521520099540A
:100F1000634AAA219954B4E0AB68A3420ED16C692C
:100F2000291C49310B22201C01F0A7FE0823201C9C
:100F3000F022E37220305B49520008E00133A34203
:100F400008D1584980239B006869C918321C01F0F8
:100F500094FE96E02B6A9C4275D3E9695A18944234
:100F600071D29C4204D168694F49042201F085FE88
:100F70004E4B1B680193022B00D082E03A6A7D69D8
:100F80004B4E944225D1C020C001FFF77DFE494B56
:100F9000019904221970484B30601A80474B012296
:100FA00004351A6015E07A698021890053189D4242
:100FB00067D2414A281C1488211CFFF7DBFE3E4BF8
:100FC000013433491C800B78019A5B02D31A051C4B
:100FD000336033682E4901930B78019A5B029A4281
:100FE000E1D2364E3368002B4BD07B6980218900DB
:100FF0005B189D4245D22F4F2F4C387803281BD8C1
:1010000003F01EF9020A131823880F211943281C24
:10101000FFF7B0FEFF2306E02388FF211943281CB9
:10102000FFF7A8FE0F23038006E0281C2449FFF7E2
:10103000A1FE01E0224B2B80224A00233360138063
:1010400023803B701DE0FB689C421AD3E41AA12266
:101050006402D2011C4BA4189C4212D81B4B786925
:101060001968002909D0F82212028023121B9B0064
:101070009A4200D91A1C211C69E78022920001F0D3
:10108000F3FD0020FEBDC04664060020CD460000F2
:101090008F060020D6460000B8080020DF4600007A
:1010A000FF0100005E0000200A4600004000002012
:1010B000600400203800002018FEFF1F34000020CC
:1010C000FF0F000008FEFF1FFFF700001CFEFF1FC0
:1010D000F8B51A4D002128780A1C01F0B9FE184E07
:1010E000184F041C3368002B1FD0174B9C4216D995
:1010F0003868FFF775FE00280DD1144B80221B685D
:1011000028785969920001F0A3FE114BE4183B685E
:10111000A4B201333B603368013B3360E2E72878D7
:1011200040210C4A01F0CEFC06E00C2CF7D92878BF
:1011300009490D2201F08CFEF8BDC04630000020A8
:101140004800002028000020FF01000004FEFF1FCF
:1011500000FEFFFF75100000C0F8FF1F38B5324BCE
:10116000041C1A680723002A5CD13048211C042281
:1011700001F0A9FE0423002854D12D4A617B126896
:1011800000294FD1A17B0139C9B20F294AD8E37B8D
:10119000217BDBB27F2916D9232B19D006D8122B3D
:1011A0003FD01A2B09D0032B2AD13AE0282B0FD09D
:1011B000A82B0DD0252B23D133E0231C0F335A78D5
:1011C000520918D01CE01E2B2BD00ED92A2B0FD180
:1011D000118B88220723114224D1164BF0221A705A
:1011E00002229A703A221A730AE0002B19D007E003
:1011F000AA2B05D1ECE79A783F2313403F2B10D060
:101200000D4D211D0422281D01F037FD281C211C35
:1012100008300831042201F030FD01232B73042330
:1012200000E00723181C38BD2C000020C245000038
:1012300004FEFF1F4C000020C0F8FF1FF7B5574BFE
:101240005749DB68051C0193564BDA7A002A4DD0CA
:101250000F2A49D0202A47D00220024244D01A78CF
:10126000E52A41D0587D1A7D9C7E00061204104369
:101270002043DC7E0F27240220434B4C019E0219A1
:10128000D2009219954202D30832954243D34400CA
:1012900024180726E4083040A200013852580628D6
:1012A00005D802F0CDFF06080F11131C1D00120512
:1012B00016E0120214E00134A4000859120E38405E
:1012C00000020AE012040BE0120109E00134A4005C
:1012D0000859FF242040120F0001104301E01203BF
:1012E000100D324A9042C8D12033AEE7304A11780F
:1012F000131C7B2911D1101C4A3000787D280CD199
:101300005078002809D1D078002806D152790320DE
:10131000002A41D001E002203EE01A7A4D2A1AD17B
:101320005A7A612A17D19A7A632A14D11A1C543234
:101330001278412A0FD11A1C55321278542A0AD138
:101340001A1C56321278542A05D11A1C57321278B8
:101350000420522A20D058789A78000212040243BE
:101360001143DA78134812061143134A09189142BF
:1013700011D8587999791A79000209040143114367
:10138000DA790E4E12060B1C13430D4A9B190020EE
:101390009A42404100E00020FEBDC04664060020A5
:1013A000B80600205E000020FEFFFF1FFF0F0000B8
:1013B00021FEFF1FFF0700E0FF1F00007F9FFFFFD0
:1013C0007F9F0000F7B55E4F041CFD680195A842A1
:1013D0006BD35C4D5C4E2A685C4B012A3DDC327855
:1013E000002A00D196E0012A0CD11D68002D00D101
:1013F000A4E000221A60FFF721FF012800D09DE041
:1014000002233370019D524A611B8918514AC1233E
:101410001568DB014902C8184F4B002D02D1196035
:10142000012111601B68C01A4C4BC2184C4B9A42E8
:101430000AD8F82212028023121A9B009A4200D97D
:101440001A1C484901F0B4F975201E21032201F04D
:10145000DFFE3C4D01232B6051E03278002A4ED054
:101460001B68002B4BD0FFF7E9FE01280BD1C020F1
:1014700098210902C00101F086F90023201C2B608D
:10148000FFF7A0FF5AE0012801DC374B1C6037480A
:1014900034494B2201F017FD002830D1344B012292
:1014A00034481A6001F0F6FC29E0BB68984207D086
:1014B0000133984223D1304880229200801800E006
:1014C0002D4880222749920001F0D7FB1D4D2B6843
:1014D000022B14D120E020338B4205D01E78DA7A1B
:1014E000E52E1FD0202AF6D1FFF7CEFB061E06D12F
:1014F000C0209821C001090201F045F92E603B6A25
:101500009C4205D180221D481649920001F0B5FB8E
:101510000E4B00221A6011E0174B80229200181C1B
:101520009918DBE7202ADDD1C0209821C0010902EB
:1015300001F029F9054A00232B6013600020FEBD4D
:101540006406002040000020440000203C000020F1
:10155000FFFF7F0014FEFF1F24000020809FFFFF7D
:101560007F97000021FEFF1F0CFEFF1F8246000038
:101570001CFEFF1FEB4600005E000020B8060020A6
:10158000F0B5C34F807B3D78ABB001900AAC002D25
:1015900040D1C04B02200126291C0A936074752398
:1015A000221C0520A573E580A580A374668126749E
:1015B00001F03AFB4023A381B74B387002210A9314
:1015C00080278023BF00DB00221CA1730520291C7B
:1015D000E380E673A780278101F026FBAF4BB04D77
:1015E000187080231B012B61A0232B83AD4B2F850B
:1015F0006B61301CFFF7F4FBC021C901AA4B0A68DC
:101600001D60013206D0A948802201F036FBA84BAC
:1016100002201860A74F0198211C052201F068FAEA
:10162000002800D19FE0E578012D05D0002D30D0B5
:10163000752D00D184E0EEE72379CB2B21D007D89C
:10164000CA2BE8D10220002102F0D4FA9A481DE00A
:10165000CC2B04D0DD2BDED1FFF73AFDDBE70026F3
:10166000311C042295483E6001F0FEFA944B9548E7
:101670001E60954B311C2A1C1E6001F0F5FA934840
:1016800004E0281C002102F0B5FA914801F002FCA8
:10169000C1E72379022B0AD0032BBCD1291C281CBB
:1016A0002A1C01F085F8291C804B0A200EE001213C
:1016B0000A1C844801F0D8FAADE7DA7A0F2A09D17A
:1016C00000290AD02035202A0AD020331A78E52AAA
:1016D000F3D113E0024211D1F2E7191C2025F2E701
:1016E00003229A76802D0BD92B1C213B5B095A1CB7
:1016F0005201203D5B018918ED1A01E00021E4E769
:10170000C020C0012A1C01F053F87F2D0DD8002104
:10171000202202A801F0A8FAC021C90168182022DD
:1017200002A901F045F82035EFE70020011C021C5A
:1017300001F03EF85E4B02221A6001F0A3F86AE75E
:101740006946227901982D3101F0D2F96379FE2B97
:1017500000D060E75F4801F09DFB281C2821022291
:1017600001F056FD57E74D4D524F287801F0D0F962
:10177000002800D145E13E682878002E26D0524E40
:101780005549336880229200C918D31A9AB201F0E1
:10179000AFF93A68131A3B603368C0184F4B30609A
:1017A00098420FDD4E4B1868421C1A60FFF70AFE84
:1017B000386800233360984204D07520042101F07A
:1017C000F1FC1EE139680029CFD114E1211C8022EF
:1017D00001F08EF943480BA90422043001F04DFAC0
:1017E000404A28780121167256729672D672167384
:1017F00001F0A0F92C4B1E68E37B032B04D03A4880
:101800003A49122201F039FA227BE37B7F2A00D881
:10181000BAE0232B00D18EE00AD8122B24D01A2B49
:1018200027D0032B00D0E6E028782F491222E0E0F1
:10183000282B5FD0A82B5DD0252B00D0DBE068469D
:101840000022336902734273328D013B110AC27365
:101850001A0E02721A0C42721A0A81738272C372D1
:1018600002A928780822C4E0237C5B0900D1BDE0EE
:1018700094E002A81E49042201F0FFF9338BD80638
:1018800002D5802369468B72287802A90422B0E031
:1018900031000020B90C00005D1100003000002074
:1018A000640600206404002004FEFF1F5E00002088
:1018B000400000202C0000201E4700003C000020BB
:1018C000480000204400002010FEFF1F02470000D7
:1018D0000E4700002B47000021FEFF1FFF01000004
:1018E00028000020C0F8FF1F4C00002070460000B8
:1018F000BE450000617CA27C090612041143227DD2
:101900001143E27C120211433F4A1160A07D3F4A1D
:10191000E17DA82B09D1637D00041B061843237EBB
:1019200018430B02011C194301E00002014311603E
:10193000FFF7CEFB19E7A37DE27D1B021A4301925C
:1019400002A80C22324901F098F9338B8822134205
:1019500011D0990603D502236A46137402E00123CD
:1019600068460374336969461A0ACB738A731A0C82
:101970001B0E4A730B73019B28781A1C0C2B00D981
:101980000C2292B202A934E02A2B0BD0AA2B09D048
:10199000002B30D1328B88231A422CD11D480123D1
:1019A000037328E0617CA27C090612041143227DA6
:1019B0001143E27C12021143134A1160A07D164AC2
:1019C000E17DAA2B09D1637D00041B061843237E09
:1019D00018430B02011C194301E00002014311608E
:1019E00011684B0213600D4A1360BEE628780C495B
:1019F000242201F02DFA287806490D2201F028FA58
:101A0000B3E62BB0F0BDC0462800002048000020FF
:101A10002C460000C0F8FF1F2C0000203C000020D6
:101A2000E64500001223038000487047414600004D
:101A30002023038000487047C645000000B50528F4
:101A400005D8044B8000C05803780B8000E00020CC
:101A500000BDC04654460000F0B50168244AA1B05C
:101A6000071C8E18C588848800216846802201F0F2
:101A7000FBF8B9686846002900D11E490B2201F025
:101A8000FCF8694618230B732023CB7203238B7653
:101A9000330A0E774B77330C360E8B77CE77002DCB
:101AA00001D1C025ED01002C00D1134CEAB26B46E8
:101AB0002D0A69469A75DD75C020E3B2240A4C767A
:101AC000CC748A734C740B768B74CD730B74C00119
:101AD000802200F06DFE041E04D1211C221C00F0A7
:101AE00067FE01E001246442201C21B0F0BDC04625
:101AF000809FFFFF38470000354600007047000018
:101B000070B50F4D0F4A2B781178DBB21940161CB7
:101B10008A060CD50C4A0D4C907823780221184087
:101B200001F046FD2B78DBB21A0700D52278327817
:101B30003F218A431A4202D0022001F08FFD70BD7E
:101B400004C0064003C006403009002007C006401C
:101B500070B50F4D0F4A2B781178DBB21940161C67
:101B60008A060CD50C4A0D4C507823780121184078
:101B700001F01EFD2B78DBB21A0700D522783278EF
:101B80003F218A431A4202D0012001F067FD70BD57
:101B900004B0064003B006403009002007B00640FC
:101BA00070B50F4D0F4A2B781178DBB21940161C17
:101BB0008A060CD50C4A0D4C107823780021184069
:101BC00001F0F6FC2B78DBB21A0700D522783278C8
:101BD0003F218A431A4202D0002001F03FFD70BD30
:101BE00004A0064003A006403009002007A00640DC
:101BF00072B6024B1A6801321A607047D40800208E
:101C0000044A00B51368013B1360002B00D162B693
:101C100000BDC046D408002008B58022044B9204C1
:101C20001A60FFF7E5FF01F02DFBFFF7E9FF08BDA4
:101C300004ED00E0F7B51E4D2B68002B0FD11D4BB6
:101C40000124A3431C1C3C3401941B4CE71A1E883E
:101C5000DE53019E0233B342F9D101342C60174E9A
:101C60003378164C5BB2002BFADA267830231E420A
:101C700000D02370124B1870062801D009280CD10F
:101C8000104B0E0C1E70104B0E0A1E700F4B19706D
:101C9000062802D112680E4B1A60FFF7A9FF2B68C5
:101CA00006489847FFF7ACFF207831231840FEBD67
:101CB000EC080020CEF8FF1FF408002000000240CE
:101CC00007000240060002400500024004000240F6
:101CD00008000240F7B50E1C0090171C1D1CFFF7F2
:101CE00087FF00980C2358432C4B2D4C196801900A
:101CF0000A18A2609268530602D42B1C103301E02C
:101D00002B1C183363600433E360301C7968009A3D
:101D1000231C01F0AFFF061E032E06D0042815D0A9
:101D2000012828D1FFF76CFF36E0A3686168586886
:101D300080221043086058684021484058609868E5
:101D40004140996039680A433A6022E0009A002ACB
:101D500004D184232B61AB61101C09E0009802F0D0
:101D600061FA104B1A684301D31884221A619A61F0
:101D7000082102F04BFA094B01981A680A4B121815
:101D8000916820680B400343802119432360396028
:101D90001360FFF735FF0026301CFEBDD008002081
:101DA000D8080020C00800200800FF03F7B5A14FA5
:101DB000A14D3B782C781C4000D13AE10823201C2F
:101DC000984300D18FE0FFF713FF012004424BD06E
:101DD00098499A4A33230B701378022633431370C1
:101DE0002B7830218B432B70954B196840238F68DB
:101DF0009F4300230B608F601178B1431170914AAB
:101E000091491370914A087013709148914A137068
:101E100013700370904803709048037090480370EB
:101E20009048037090480370904803709048037086
:101E30001370904A1370904A1370904A13700423E1
:101E40000E781E40FCD18E4B8E4A1B688E4F9A60D6
:101E50008E4A04201A60311C321C3B1C01F00AFF20
:101E6000794B0D22BE741A70A00717D5884B1A78CB
:101E7000510705D5874A874F5268019201327A602F
:101E80001A78900705D58349824F09680A1C0132E8
:101E90003A60062267481A7002230370E1060CD5E7
:101EA000644A302313702B782022134300212B70B7
:101EB00005200A1C0B1C01F0DDFE20231C420BD068
:101EC0005C4F30223A702A7800219A432A7006200B
:101ED0000A1C0B1C01F0CEFEFFF792FE0823201C0B
:101EE0005449984308700820044200D15FE76A4AC9
:101EF000634B14781968240916786301CB18624D76
:101F000006421FD00C2262434D4909688A18AA6014
:101F10009268570604D41A1C10326A60143303E026
:101F20001A1C18326A601C33EB60FFF761FE221C3A
:101F30002B1C0021032001F09DFEFFF761FEAA7C0F
:101F4000404B69E01078042210401A1C002801D090
:101F500008324020286010688601B60D2E823C268B
:101F60003040042802D0342825D057E00C256543A2
:101F7000334E8027306841198868000701D5096809
:101F80000F403148A10009180978C80602D5201C65
:101F9000012101E0201C0221FFF79CFE33685D193E
:101FA0008023002F03D0296899430B1C01E02A6885
:101FB00013432B6039E02F6800200C2618619861CC
:101FC0001F4D364866437F0608D42F68BE19B66891
:101FD0003040C02608603043886007E02F68BE1993
:101FE000B6683040C0268860304308600C266643DF
:101FF0002868811948204860201C0021FFF76AFEEC
:10200000012805D02B689E19316880230B4333606B
:102010000A4B20211A788A431A7006E084221A613A
:102020009A61201C082102F0F1F8024A082313707B
:10203000BDE6F7BD8020074084200740942007407C
:10204000D008002098200740C0200740C420074047
:10205000D0200740C8200740D4200740D8200740A0
:10206000DC200740E0200740E4200740E82007404C
:10207000EC200740F4200740F8200740FC200740F0
:10208000C008002088000800D8080020C800080008
:1020900088200740C4080020902007400800FF0364
:1020A0000E4B10B51B6884004033E2500C4A890186
:1020B0008318C9B21970C317DB0E1B18094A5B11CC
:1020C0009B009B18084A104004D520220138524238
:1020D00010430130012282401A6010BD08ED00E07B
:1020E00000E400E000E100E01F000080074A084B28
:1020F000DA63084A084B1A60084BC0221968920438
:102100000A431A60064B07221A607047191C000028
:1021100000F8FF1FFF9E240014E000E020ED00E027
:1021200010E000E0074B00B51A680C231A4204D0F7
:10213000054B55221A60AA221A60044B20221A600D
:1021400000BDC04600810440048104408CF00F4073
:10215000134B021C196880239A43530140B210B5F7
:10216000CB18002813DA0F48910009180C204243BD
:102170000D4800688218546840208443546000224F
:102180001A619A610B78022293430B7006E019687A
:1021900098680422914390431960986010BDC0462E
:1021A000C0080020C0200740D008002038B5184AD9
:1021B0000C1C18491568820052181278031C012063
:1021C000510723D50C225A4313495B010968ED18C6
:1021D0008A18A260FFF70CFDA3689B685A0604D416
:1021E0002B1C10336360143503E02B1C1833636021
:1021F0001C356368E5601C6880231C4003D0FFF732
:10220000FFFC022002E0FFF7FBFC201C38BDC046AB
:10221000C0080020C0200740D0080020F0B59C4630
:10222000384B394D1C688B005D19161C4B012A7800
:10223000E4180C239A432A704B43344A85B0116842
:1022400000270393CB18A7612761A7602760029539
:102250009F601F602E4BFF2805D11A7830218A43DA
:102260001A702F704CE01978102529431970051C3D
:1022700080239D4301951368012D04D1039D5B19B3
:102280005F60242505E0039D08225B195A6005253F
:10229000482740B200282EDB616800290CD1331C8E
:1022A000664500D263469EB2301C00F045FE606079
:1022B000301C00F041FEE060164B31040B401F4320
:1022C0008023191C3943A16040218F433B43236085
:1022D0000E4B03991B6808225B189F60019B2A43E1
:1022E000002B01D1151C03E004239D4318231D433B
:1022F00002990D7004E0019A002AF9D01023F6E744
:1023000005B0F0BDC0080020C0200740D008002064
:10231000842007400000FF03F7B50C26184B464306
:10232000184F1C6839684301E4188B5940252B422B
:1023300002D00022009201E0083400952268802536
:10234000131C2B40019301990123002916D19201FE
:10235000920D616801F010FC022301280ED03B6849
:1023600000999E19B268084B13400B432A1C1A436C
:102370002260326815402B433360019B181CFEBD60
:10238000C0080020D00800200800FF03F7B5484A25
:102390004B7C10680C1C474901330140802000062B
:1023A00001431160227CDBB2012A05D1424AA021FF
:1023B0001068C902014308E0404A80211068890181
:1023C00001431160E0213E4AC90011603D4A80216D
:1023D0001068C902014311601D1C102B00D9102583
:1023E000EDB20C20684300F0A7FD374E374B30604C
:1023F000197880220A431A7034490B785BB2002B9B
:10240000FADB334F022380213B706801994000F0D2
:10241000B7FD304D304B2860000A18706A882F4B8A
:102420001A70EA782E4B1A702E4A002313702E4A27
:102430003B7013700423117819400191FBD10820DF
:102440002F6800F079FD786008202F6800F074FD97
:102450002B68264AF8609A60254A18201A6033686B
:10246000244A03219A60204B0D221A70224BED2240
:102470001A70224BFF221A70214BBF221A70214A78
:10248000FFF70EFE019A204B11481A701F4B8B224A
:102490001A701F4B06221A700123037062891A42B8
:1024A00005D00A4940230B701A4B10221A70F7BD51
:1024B00000700440FFFFFFBF0480044038800440E8
:1024C00068D0044034800440D00800200C2107402C
:1024D00094200740C00800209C200740B0200740FF
:1024E000B420074098200740C0200740880008001B
:1024F000C80008000800080010200740802007409E
:1025000088200740AD1D00000021074084200740BF
:102510008C2007400821074000B5084B8000C358B5
:1025200001201A7952B2002A06DAD9718022D978AC
:1025300052420A43DA70002000BDC046D447000072
:10254000034B8000C3587F22D9780A40DA70704765
:10255000D44700001C4B820010B5011CD458012840
:102560001ED000280ED0022829D1184B80221868CE
:10257000520102431A60C022154B92001A600E20CD
:10258000144A1AE0114B80221968D2000A431A60DB
:10259000C022114B92001A600C2002210F4A0CE05D
:1025A0000A4B8022196892010A431A60C0220C4B20
:1025B00092001A600B4A0D200221FFF771FDE378AB
:1025C00008221343E37010BDD44700003880044054
:1025D0000CC00440011B000044A00440A11B0000EB
:1025E00000D00440511B0000034B8000C358372229
:1025F000D9780A40DA707047D44700001C4B82003B
:1026000010B5011CD45801281ED000280ED0022875
:1026100029D1184B80221868520102431A60C02247
:10262000154B92001A600E20144A1AE0114B8022BA
:102630001968D2000A431A60C022114B92001A6036
:102640000C2002210F4A0CE00A4B802219689201EB
:102650000A431A60C0220C4B92001A600B4A0D20EC
:102660000221FFF71DFDE37824221343E37010BD20
:10267000D44700003880044008C00440011B00001B
:1026800040A00440A11B000004D00440511B0000E6
:10269000034B8000C3582421DA788A43DA707047EC
:1026A000D44700002D4B820070B5D358012819D0B3
:1026B000002807D0022850D1294A802416686401D6
:1026C000344314E0264A80241568E4002C43146047
:1026D000244A254C166834431460CA790B2A0DD954
:1026E0009D220EE01E4A8024156824012C431460AC
:1026F000CA790B2A2FD852001C4C01E01C4C520006
:10270000125BD404E40ED2B21C705A700A88194DC0
:102710000624D6070AD57F262E54144010D054071D
:1027200001D5032200E002229A700AE0FF262E540F
:10273000144005D0550701D51322F5E71222F3E71F
:102740009C70002809D00A88D60606D51A78202160
:102750000A431A7001E04E22D3E770BDD44700004F
:10276000348004400480044000000104A2470000BB
:10277000BA4700003009002008B5002144200A1C97
:10278000FFF758FA08BD38B5840A4518A402092095
:10279000211C0022FFF74EFA002806D180232A1BB5
:1027A000DB009A4202D9E418F1E7012038BD0000AD
:1027B000F7B503230191161C204C002909D122688A
:1027C0001A4201D1002038E09A432260042200928C
:1027D00004E0021C9A43184022600090009B0425EC
:1027E000ED1AB54200D9351C154A009B0199D7183E
:1027F000381C2A1C00F041FA019A114B52197F191A
:1028000004330192761B9F4210D3062021680C4AA4
:10281000FFF710FA051E0FD1236809480433FF2182
:102820000422236000F020FA009502E023685D197D
:102830002560002ED2D1C5E70120FEBDCC080020C6
:10284000F00800200C4B30B5C0180003002A03DA52
:102850000A4B03241A4000E0094C0123E4430029F9
:1028600009D0194204D005689943254015430560F5
:1028700004305B00F3E730BD490004008BF8FF7FB4
:1028800077070000024A034B00B51A60FEE7C04616
:102890000400FA050CED00E010B5124A1249134885
:1028A000891A00238B4203D0C45CD4540133F9E766
:1028B0000F49104A914205D10F4A10490023891A45
:1028C000181C08E00E480023801A8342F4D0CC5C28
:1028D000D4540133F9E78B4203D0D418207001336C
:1028E000F9E710BDC0F8FF1FDBF8FF1FE447000049
:1028F0001004000010040000DCF8FF1F7009002025
:1029000008430000424B80221968D2000A4310B5E8
:102910001A60404A03201168814311603E493F4AD2
:1029200011603F4A1168022211403E4A00D00C213A
:1029300011603D4A082111701968802212010A4372
:102940001A60A222202152000220FFF77BFF374BA2
:1029500020221968364C11431960364B19680A4316
:102960001A60354BA4221A70344BA0221A7002212F
:102970001A1C20782E4B0842FBD0102118780842F0
:10298000FCD10C20197801400829FBD12C492720C3
:1029900008702C4958200870202118780842FCD073
:1029A000402118780842FCD027492848086028218F
:1029B00011700C211A780A400C2AFBD1244B254AAD
:1029C0001360254ADA601A615A619A611A639A6043
:1029D0009A63DA62FFF760FF204B214A1360214AB5
:1029E0001360214B1A6805221A608022520219686E
:1029F0001142FCD0FEF71AF91C481D4900F07EFA7E
:102A00001C481D49092200F0E1FA00F097FBFCE7A1
:102A10003880044054F00F400301030080A00440BC
:102A200050F00F400081044002D0074080F00F407A
:102A30000640064094F00F4001400640004006402A
:102A40000440064005400640448004400000011058
:102A500000F8FF1F08ED00E0FD1A0000FFFFFF0077
:102A600014E000E018E000E010E000E0444700005F
:102A700070090020544700004C47000001688D4653
:102A8000406880477047000013B5441E0548E4B213
:102A900000682301C318187B00941C680323A04717
:102AA00016BDC0463409002008B5044B187000015B
:102AB00000F042FA024B186008BDC04633090020FE
:102AC0003409002037B5031C0D1C0020FF2B0CD04F
:102AD0000648013BDBB2046819016418207B0093AF
:102AE000111C24682A1C0223A0473EBD3409002083
:102AF00013B5441E0548E4B200682301C318187BCF
:102B000000941C680423A04716BDC0463409002069
:102B100013B50749421E0968D2B21301CB18187BBE
:102B2000002100921C680A1C0523A04716BDC04660
:102B30003409002013B50A1C0649441E0968E4B292
:102B40002301CB18187B00941C6800210623A047A2
:102B500016BDC0463409002030B50A4B0A4A1B682E
:102B600014780022A2420BD01D680132854204D1A4
:102B70001D7B8D4201D1D0B203E0D2B21033F1E718
:102B8000002030BD3409002033090020F0B5061CB8
:102B900085B0101C019102920393FFF7DDFF011E27
:102BA00001D000203AE0FFF7D7FF071EF9D01C4BF9
:102BB000C5181C4B2D011B685D193388002B13D0E1
:102BC000039800F0B9F9041C68600DD03388181C14
:102BD000009300F0B1F90028E3D0009B2060606012
:102BE000A060C018E060E3827388002B11D00398C6
:102BF00000F0A2F9041CA8600BD07688301C00F00D
:102C00009BF90028CDD020606060A0608019E06052
:102C1000E682029B381C2B60019B2B7305B0F0BD34
:102C2000FFFFFF0F3409002007B5032807D0052850
:102C300011D0002813D1101C00F05EFC10E01389A5
:102C400001A80380002343801368064A19781823DB
:102C5000FFF79CFF04E0101C00F030FF00E00020B4
:102C60000EBDC046012D000000B5031C8218934222
:102C700002D019700133FAE700BD10B5002393426A
:102C800003D0CC5CC4540133F9E710BDF7B5038A17
:102C9000041C0E1C4768151C9A4200D91D1CADB2BD
:102CA000002D28D0E3687A1962609A4215D3DB1BA5
:102CB0009BB22268E91A0093531863600191FEF7F2
:102CC0009FFF002E12D0391C009A301CFFF7D5FF51
:102CD000009B2168F018019A06E0FEF791FF002E94
:102CE00004D0301C391C2A1CFFF7C7FFFEF780FFF9
:102CF000238A5B1B2382FEF783FF281CFEBD000096
:102D0000F7B51D1C174E08AB1B78019131681B01EC
:102D10000093CB18171C5C68FEF76AFF052D09D0DD
:102D2000062D09D0042D16D1201C01993A1CFFF75D
:102D3000ADFF16E0258A11E0012F03D13368009A18
:102D40009B189C68002C08D02368258AA3606360C8
:102D50000023238202E0002500E0251CFEF750FF3F
:102D6000281CFEBD34090020F7B5041C151C0F1CDF
:102D7000FEF73EFF218A628AE38A8818401998424A
:102D800002DD5D1AAD1AADB2A168AA186282019186
:102D90004A19E168A2602E1C8A4205D3D31A226820
:102DA000A3609B1AEE1AB6B2FEF72AFF0198391CEF
:102DB000321CFFF762FFB54204D0B919AA1B206884
:102DC000FFF75BFFFEF714FF638AA28AAB4206D1CE
:102DD000238AEB189A1800232282A38202E0AA1801
:102DE000A2825B1B6382FEF70BFF281CFEBD000066
:102DF000F8B502784378041C0F1C00259A421ED1B6
:102E000086781048311CFFF7A7FEA84217D00E4B5A
:102E1000C0180E4B00011B681818E3784068032B9C
:102E200004D1C58A038AED1AADB208E0211C3A1C10
:102E3000FFF79AFF0421051C70B200F0B3F9281CBB
:102E4000F8BDC046012D0000FFFFFF0F3409002030
:102E500008B5031E04D1081C111CFFF7C9FF05E0CB
:102E60000020FF2B02D0181CFFF70EFE08BD38B55E
:102E7000041C031C1A1B0133581E057892B2002D46
:102E8000F8D1281C002A03D0081C211CFFF7E0FF02
:102E900038BD000008B5024B1978FFF7E8FF08BD00
:102EA000DAF8FF1F07B5031C002083420AD06A46E8
:102EB0001070507093701171012368460521D37012
:102EC000FFF796FF0EBD30B50023934208D0C45CD7
:102ED0000133CD18013D2D78A542F6D0012000E048
:102EE000002030BD10B5031C0C78181C1C700A782B
:102EF000013352B20131002AF6D110BD0A4B10B590
:102F000000221A80094B0A4A19600A4B147819608A
:102F10001A1C0378A34203D0002B04D00430F8E736
:102F20004388C918116010BD3C09002038090020F1
:102F3000CDF8FF1F40090020F8B50E4F0E4E3B683C
:102F40003488051C1C1903231C4201D09C43043403
:102F50000A4A631912689A420AD92A1C201C0021C5
:102F6000FFF782FE3B68201CE31AED18358000E075
:102F70000020F8BD380900203C090020400900204D
:102F8000F8B50F4F0F4E3B683488051C1C194B1EBB
:102F90001C4202D04B421C4064180B4A6319126851
:102FA0009A420AD92A1C201C0021FFF75DFE3B68CB
:102FB000201CE31AED18358000E00020F8BDC04663
:102FC000380900203C09002040090020F0B585B0F8
:102FD0000392554F554A002313603B60544B061C27
:102FE0001B780C1C2578002D48D06DB29D423ED137
:102FF000221CA31ADBB20293013400256557002D71
:10300000F7D1142058430430FFF796FF0299386037
:10301000CB43E4182F1C6178002926D049B2331C19
:1030200001911A68002A1ED0002151568C46019940
:103030008C4516D15968026041601A890281002AC4
:1030400001D00135EDB2598941819A8982819B7BFA
:10305000C373002901D1002A01D00137FFB2143017
:1030600001E01033DDE70134D5E7016008E0013409
:103070000022A256002AFAD10134B3E72F1C029590
:10308000294C2368002B47D0002F2BD00C207843ED
:10309000043080B2FFF750FF244E264A2368306088
:1030A00094461A68002A19D05A89002A06D0624527
:1030B00001D1002159815A89426003E09989002990
:1030C00001D0416001224168002901D001214172F3
:1030D000002A01D003600C301433E2E70C235F4375
:1030E000C01B3060039BE818C0B2FFF7DDFC002D69
:1030F00012D02468216800290ED02389002B09D022
:1031000003200121221CFFF78FFDA073002801D1AD
:10311000FF23A3731434EDE7074B00221A60FEF778
:10312000E5FF029805B0F0BD440900204C090020DD
:10313000CDF8FF1FFFFF000048090020184B37B5EE
:103140001C682368002B29D0E27B0D231A4223D070
:10315000FEF74EFDA389002B02D1E37BD90716D4DD
:10316000237C002B0ED000256A461570557021680F
:10317000281C0A7869468A700522CD700B71FFF70A
:1031800067FE2574E27B0A23134000D1E373FEF748
:1031900037FD201C626890471434D2E737BDC04623
:1031A0004409002038B5174B1C682368002B27D032
:1031B0001B785BB2834221D1002918D1124B1D68C4
:1031C000002D14D02B68002B11D09C420DD1FEF79E
:1031D0000FFDA389002B03D00C4A12689B186B606B
:1031E0000023E373FEF70CFD0AE00C35EAE74A071B
:1031F00002D5E37B1A0703D4E17301E01434D4E76A
:1032000038BDC046440900204C0900204809002070
:10321000F8B5194B0E1C1C68171C002C2BD0174B33
:103220001D682B68002B26D01B785BB2834220D10F
:103230002368002B1FD09D4219D1FEF7D9FCEB7BF0
:1032400002229343EB732772002F04D1AE81002E2C
:1032500004D1667208E0002E00D10126084B1B68DD
:10326000F618012366606372FEF7CAFC03E00C34B3
:10327000DEE71435D5E7F8BD4C09002044090020ED
:1032800048090020144A154B11681B680131F0B53C
:10329000101C1160002B1ED00224082504261A6879
:1032A000002A18D0597A002913D001685F68B94202
:1032B0000FD1D17B214204D1294200D1D673197A92
:1032C00011749289002A03D059688A185A6000E064
:1032D0005A720C33E3E7F0BD480900204C09002086
:1032E00038B5051C2020FFF727FE041E01D1002061
:1032F0000BE0281CFFF720FE20600028F7D04319C0
:10330000A0606060E360E582201C38BD10B50B7FD3
:103310000C1C9A070FD01121DA0700D41321FFF7F4
:10332000FBF8C0B2002825D1237F0322934340221B
:10333000134323771EE09A061AD40A8A002A03D17F
:10334000402293430B7713E04B681978FFF7E4F8BA
:10335000237F4022134323776368E268013363606D
:10336000934201D323686360238A013B238201E0F7
:10337000FFF7E6F810BD0000F7B51D1C08AB1B7881
:10338000071C0191141C0093FEF732FCA81E0428B0
:1033900000D9A7E00099564E0D0100F051FF033609
:1033A000592B80003368019A5D19D20401D5AD68AC
:1033B00000E06D68002C1BD0E30703D5381CFFF735
:1033C0001DF904E0A00702D5381CFFF761F9610779
:1033D00003D5381CFFF7BEF804E0220702D5381CDD
:1033E000FFF702F9630603D501987F2303406B774B
:1033F0006D8B78E033683F4A5D196B68598B1142D9
:1034000001D01D8B6FE01D8A6DE0336801995D1955
:10341000AD68002907D1EA8A2B8A0D1CD31AA34272
:1034200061DB9DB25FE0FEF7EBFB221C0199281CDB
:10343000FFF79AFC041CFEF7DBFB2A7F60231A428D
:1034400003D1381C291CFFF761FFFEF7D9FB4DE0C3
:103450003268019953195B68221C181C0093FFF70E
:1034600015FC009960224B8B041C13423ED00A7F4E
:1034700010210A423AD00098008A132836D88A438D
:1034800000990A779A0631D5336801225D19A96837
:10349000381C0B7F13430B77FFF738FF26E03368A8
:1034A000002C02D05D19AB6815E05A195368102042
:1034B000197F01420FD08143197791684B8B980691
:1034C00006D50B7F012213430B77381CFFF71EFF35
:1034D00033685D196B681A6800259A605A601D820E
:1034E0001D8300E00025FEF78BFB2C1C201CFEBD7D
:1034F000340900208080FFFFF7B5284E041C0F1C04
:103500008179301CFFF728FB051C0190002D02D0AB
:103510007A0707D441E0291CFFF71EFB051C019820
:10352000002D3AD01E4B1D4AEE181E4B36011B686B
:103530009E193260BB0709D5A279A0880192FFF7D6
:10354000CFFE019AB0609300174AD050FB0707D511
:103550006088FFF7C5FEA379144A9B00D0507060C5
:10356000A379114A9B00D358002B01D022885A839B
:10357000A3790E4A9B00D358002B07D0227A5A77A2
:10358000A3790A4A9B00D35822885A83A379211C25
:103590003373A079FFF786F8281CFEBD793300004D
:1035A000FFFFFF0F340900205C09002050090020B4
:1035B00038B5021C8B00081C25495C582549658BD1
:1035C000595820231D420FD0132A03D10A7F1343D9
:1035D0000B773CE0112A07D10A7F1A4237D09A4371
:1035E0000A77FFF793FE32E0238AE58A9D420BD9E2
:1035F00001332382A3681A70A368E5680133A360CE
:10360000AB4201D32268A260638B6022134213D0C5
:10361000227FD50610D4E58A228A133D95420BDC21
:103620009A0605D50B7F022213430B77FFF76EFE38
:10363000237F102213432377628B074B1A4206D154
:10364000607F002803D040B20421FFF7ABFD38BDF6
:10365000500900205C0900208080FFFF08B5034B63
:103660008200D158FFF752FE08BDC0465C09002019
:1036700010B5002808D08369581DC27F541C0C3235
:1036800052009B18C477998010BD10B5831CCC07DD
:1036900006D5047814804078000204431480023276
:1036A000981C8C0706D51C7814805B781B021C4381
:1036B000148002324B0705D5037813804178090244
:1036C0000B43138010BD0000F7B5282401935C4321
:1036D000364B00901B6800201C19E38A089E834229
:1036E00062D12283131C8A4200D90B1CA28A9FB28A
:1036F000E382974201D9628200E06382F368009915
:10370000658A1960B36880205A6829041043284AE2
:10371000114072680143116059684022514059605C
:103720009968E0684A409A60291CFFF7A1FF009A57
:103730006260E28A638A9A4207D0E368002B06D06F
:103740009B690533DB7F012B01D9E08A2CE00198CE
:10375000311CFEF72BFD0028F7D17B1B9FB2009B8D
:103760005B190093A38A3D1C9F4200D91D1CF3687E
:10377000009980201960B368ADB25A6829041043DB
:103780000B4A114072680143116059684022514050
:1037900059609968E0684A409A60291CFFF768FF01
:1037A000638AEB186382C4E7FEBDC0466C09002043
:1037B0000000FF03F0B58BB01C1C10AB03900F1C76
:1037C000161C1D78FEF714FAA01E042800D995E0F7
:1037D0004D4B2D011B685D1900F032FD031A671770
:1037E0008500F80401D5AB6800E06B68710608D568
:1037F0009A69911CC97FC80703D57F210F40013208
:10380000D7779B690233DD7F79E06B681D8A76E0AC
:10381000AC68002C0CD1039805A9FEF7C7FC251C49
:1038200000286CD105A90091381C311C321C37E0EE
:10383000A36900250233DB7FDA0760D5AF4206D1EA
:10384000E28A238AD31AB34259DB9DB257E0FEF7CE
:10385000D7F9391C321C201CFFF786FA061C051C00
:10386000FEF7C6F9A36940270233DB7F3B4246D10E
:10387000039805A9FEF79AFC002840D1A269616867
:10388000E0680232431AD17F9BB20F43D777321CD4
:103890009E4200D91A1C92B205AB6068111C0093BD
:1038A000039BFFF711FF051C29E06C68391C321CD3
:1038B000201CFFF7EBF9A36904270233DB7F061C0A
:1038C0003B421FD0FEF794F9A3690233DA7FBA4373
:1038D000DA77A169887EFEF71FFD0028F9D0FEF790
:1038E0008FF9301C0EE0002E01D0AB6800E06B6851
:1038F0001A6800259A605A601D8200E00025FEF7D4
:103900007FF9281C0BB0F0BD34090020F0B58BB056
:103910006C4626340390201C049105921E1CFEF771
:1039200087F8039C01218C4662426241D2B2002397
:1039300007926F460578FA8C0195521B92B2FA8471
:1039400002924278042A12D0052A23D0022A42D1B8
:103950004379039C1B1B5A425341DBB2002B02D11B
:10396000079D002D37D000270123BC4633E0002BF4
:1039700031D0049CFF2C02D08278A2422BD1059D2D
:10398000FF2D03D0C2780323AA4224D1002E2CD0CD
:10399000022320E0002B1ED0002E1CD09D1E6A4268
:1039A0005541321C1168002912D08F7884787C40F0
:1039B0007F273C420AD1002D0DD14D7909792D0286
:1039C000294395888D4206D2918004E00832E9E7C8
:1039D000002D00D010600199029A4018002AA8D149
:1039E000644660426041404230400BB0F0BD37B5A4
:1039F0008369051C0133DB7F002B13D0028A8A42C6
:103A000010D86A46937001230024D370DD2313710C
:103A100014705470201C69460522FFF719FAAB692F
:103A20000133DC7737BD000070B5041C80780B1CB7
:103A30007F22011C114028254D430C4E9043E27813
:103A40003668104362797519267912023243FEF7FF
:103A5000E5FBE278AB1C002A01D1112203E003351B
:103A6000EA7F01210A43DA7770BDC0466C09002065
:103A700038B5011C7F23194028244C430E4B0022EB
:103A80001B68FF201C19131CE568FEF7C7FB002309
:103A9000A21CD377621DE382D3779D4203D02B8291
:103AA0002B68AB606B60A368002B04D000221A82E5
:103AB0001A689A605A6038BD6C090020F7B5051C79
:103AC000294F1C230430A97B284A3C68FFF75EF885
:103AD0000190AE7B2823002E0AD05E43AB89A41947
:103AE000A3826B89D90613D5E31C2022DA770FE075
:103AF000687C01305843FFF71FFA0823838238603F
:103B0000AA7C431C041CDA77301C291CFEF73EFCFF
:103B1000019B17495A18174B12011B689A18936892
:103B2000E360002B02D09C612B892382AB7BA376C0
:103B3000AB7B002B0CD0EB7B002B09D028245C4303
:103B400039680C19A376A97B231DD977AB89A38289
:103B50005368A360002B03D09C61AA7C631CDA77B6
:103B60002D6801982560FEBD6C090020B537000066
:103B7000FFFFFF0F34090020F0B5151C1C4A85B06B
:103B8000146828225043241827680E1C002F03D1E4
:103B9000A068002807D129E0081C1A1C291CB84776
:103BA000072823D1F4E7631CD87F002803D040B254
:103BB0000421FFF7F7FAA3680234E17FA4460191DC
:103BC000019C04210C400120002C0FD1DA8A1F8AAD
:103BD000D21BAA4206DB181C311C2A1CFFF7C4F8B2
:103BE000201C03E0019A63460A43DA7705B0F0BD72
:103BF0006C090020F0B5A1B00E1C80220021051C2C
:103C00006846FFF731F8301CFF2100226B46FFF7B2
:103C10007DFE002828D0164F00246B461859002836
:103C200023D0002D0BD1002E03D18078FFF720FF89
:103C300018E000AA13199988FFF7F6FE12E08278BF
:103C40007F231340282253433A68D31802330222B9
:103C5000D97F012D01D1A94302E091430A1C012122
:103C60000A43DA770834D8E7012021B0F0BDC04616
:103C70006C090020F0B5A9B00D1C04920393002438
:103C8000062800D9B4E200F0E5FA0A018A028302AC
:103C900007009202A302AA02049828254543C34BB9
:103CA0001B685D19EF8AEC68002F28D1002C00D129
:103CB0009EE2238A002B1BD06268E1688A4202D30D
:103CC000E08A121A62606068091A89B20A1C994275
:103CD00000D91A1C92B20399049B0091111CFFF7A2
:103CE000F3FCA269201C118AFFF781FE00247FE209
:103CF000A26940200232D17F8143D177F6E76B8AF7
:103D0000BB4200D290E0002C6FD0268A002E6CD0EF
:103D1000A3695A1D988BD17F8446012901DDD88B78
:103D200098830139D177A2696146761A131CB6B21D
:103D3000059226820533DB7F591C49005B00D018B1
:103D40004942002302911A1C0299023B8B4205D082
:103D5000C118898B8C46624492B2F5E7964230D105
:103D6000002EBED1AB1CDA7F30231A4215D0A98AAF
:103D7000381C00F0BDFA89B200290ED1039A8821BF
:103D800093685268586801260143116059684022BF
:103D90005140596099684A409A606268E368D7194F
:103DA00067609F4202D3E38AFF1A67600023EB82B9
:103DB0009E4296D1059B40210233DA7F8A43DA770F
:103DC0008FE76068E368C71967609F4202D3E18AA2
:103DD0007F1A67606068B61A1B1A99B2B2B28E4237
:103DE00000DB0A1C0023EB8275E7A98A381C00F06F
:103DF0007FFA89B2002914D12B8BBB4203D1AB1CB3
:103E0000DB7F98060DD503998B684A68586888212E
:103E100001431160596840225140596099684A40F5
:103E20009A600024EC82E3E1FF1AAB8ABFB23E1C29
:103E30009F4200D91E1CB6B2002C11D0A3695A1D96
:103E4000D17F988B012901DDDF8B9F830139D177E9
:103E5000238AA2691B1A2382118A201CFFF7C7FD3F
:103E6000039869686A8AC3688A181A608368426816
:103E70005968802008434E49370439400143116096
:103E80009868596840225140424059609A60311CFC
:103E9000201CFFF7EDFB6B8AF6186E8226E7434B7A
:103EA0000C781F6800268021FE828C43012C00D1F3
:103EB00099E0022C00D115E1B44200D05FE16878AE
:103EC000092800D983E000F0BBF97C82828282411C
:103ED00005827745E878AA78EE79AB79000210433D
:103EE00036021E43FF22031C8021934389008B422C
:103EF0000CD0C02189008B4214D080225200934202
:103F00001BD108AD281CFDF78DFD12E008AD281C63
:103F1000FDF78EFD039B29880093321C0023FFF7D9
:103F2000D3FB65E108AD1040291CFDF787FD002893
:103F30001AD0039A29880092EFE73B680424002BEB
:103F400000D155E1039A681C118A48E0AB780398C8
:103F500083748FE0A978174C00202170FFF74AFE88
:103F6000061E03D000232370042441E10F490324DB
:103F70000B680133DB7F0393002B00D138E16846E7
:103F8000A91C01222630FEF778FE08AF039A75239C
:103F9000FB700223BA703B71301CFE23391C0722D0
:103FA0003E707E707B71FEF753FF21E16C090020AB
:103FB0000000FF036A090020039B8F480093012142
:103FC00003E00398022100908C480A1CA6E73B6896
:103FD0000424002B00D10BE1039A281C118A002233
:103FE0009847041C04E16B78A81C04930A2B43D067
:103FF0000B2B02D0002B6DD15CE07F4F04243B786B
:10400000002B00D1F4E007AC0321221CFFF73DFB9D
:10401000A578311C802208A8FEF726FE3878291CD6
:10402000FF2208ABFFF772FC083608A88319083B8B
:104030001D68002D03D0A878FFF71AFDF4E7A678D5
:104040002478291C8022FEF70FFE221C3878311CB0
:1040500008ABFFF75BFC0424002800D1C8E008355A
:1040600008A94B19083B1868002803D00021FFF766
:10407000DBFCF4E70324BBE05F4F04243B78002B18
:1040800000D1B5E008AD02212A1CFFF7FEFA38780E
:1040900029780122331CFFF739FC002800D1A7E062
:1040A000039A0121009203300A1C331CFFF70CFB1A
:1040B000341C9DE0504B04241B78002B00D197E06A
:1040C000039B022100934E480A1C049BFFF7FCFA55
:1040D000049C8DE03B680424002B00D188E0039809
:1040E000018A52E069780491012940D808AEA81CE1
:1040F000211C321CFFF7C9FA3F4B1B78002B03D160
:1041000033880424002B73D130881F2228230240D7
:104110005A430499BA1802320823012915D1D17FD4
:10412000194200D1E2E599433B68D177002B00D1D9
:10413000DCE5C0B207AC2070FEF70AF8314A201C5B
:10414000136800211B6804224AE7D27F134006D07F
:10415000039B022100932C480A1C002304E00398CF
:104160000221009026480A1CFFF7AEFABEE53B6824
:104170000424002B3CD0281C0821032230E73B6894
:104180000424002B34D0039A118A281C321C27E700
:10419000039B1A8A002A02D10498022304E00398A0
:1041A000291C028A04980123FFF7E6FC19E703990A
:1041B0008B7C002B07D0134B1F201B68CC210133B5
:1041C0001856FEF76FFE0020011CFFF713FD8DE56A
:1041D0000C4B1F201B68CB210133185605E0094BFF
:1041E0001F201B68CA2101331856FEF75BFE7DE5D0
:1041F000201C29B0F0BDC0466A09002068090020D3
:10420000E24700006C090020E047000028235843E3
:10421000034B1B6818180230C37F1943C1777047DE
:104220006C0900202822034B50431B6818180430E7
:10423000C07F70476C09002008B5FDF773FF08BD0B
:1042400002B4714649084900095C49008E4402BC29
:104250007047C04603B47146490840004900095AF6
:1042600049008E4403BC7047002934D0012300224A
:1042700010B488422CD301242407A14204D28142E5
:1042800002D209011B01F8E7E400A14204D28142F5
:1042900002D249005B00F8E7884201D3401A1A4372
:1042A0004C08A04202D3001B5C0822438C08A042A9
:1042B00002D3001B9C082243CC08A04202D3001B5F
:1042C000DC082243002803D01B0901D00909E3E7D9
:1042D000101C10BC7047002801D00020C04307B458
:1042E000024802A14018029003BDC0461900000018
:1042F0000029F0D003B5FFF7B9FF0EBC4243891A7D
:084300001847C0467047C04693
:104308000D0A436865636B696E6720466C61736864
:104318002E2E2E000D0A0A57726974652D65727269
:104328006F72212120284374726C2B7220746F20C5
:10433800726573657429000D0A0A20755461736BE0
:1043480065722053657269616C204C6F6164657297
:104358000D0A003D3D3D3D3D3D3D3D3D3D3D3D3D25
:104368003D3D3D3D3D3D3D3D3D3D0D0A005B002F42
:10437800005D0D0A006D65203D206D617373206539
:10438800726173650D0A006263203D20626C616E84
:104398006B20636865636B0D0A006463203D2064CD
:1043A800656C65746520636F64650D0A006C642034
:1043B8003D207374617274206C6F61640D0A00672C
:1043C8006F203D207374617274206170706C696332
:1043D8006174696F6E0D0A3E2000112A000D0A44AF
:1043E800656C65746520636F6465205B792F6E5D0D
:1043F800203F203E20000D0A506C656173652073D4
:104408007461727420532D52454320646F776E6C2B
:104418006F61643A20000D0A5374617274696E67A3
:10442800204170706C69636174696F6E0D0A0A00CF
:104438000D0A4D617373206572617365205B792F76
:104448006E5D203F203E200020454D505459210DDF
:104458000A3E2000204E4F5420424C414E4B210D25
:104468000A3E2000203F3F0D0A3E20000D0A212170
:104478002044657374726F7920464C41534820611B
:104488006E64204C6F61646572202D20636F6E66C8
:1044980069726D205B792F6E5D203F203E20000DF4
:1044A8000A0A44656C6574696E6720636F64652EDB
:1044B8002E2E007375636365737366756C0D0A3E03
:1044C80020006661696C656421210D0A3E20000D9B
:1044D8000A41626F7274656421210D0A3E20002032
:1044E80041626F72746564210D0A00534F46545738
:1044F800415245533139000D0A0A535245432D653F
:1045080072726F72212120284374726C2B7220748E
:104518006F20726573657429000D0A0A43532D656F
:1045280072726F72212120284374726C2B7220746E
:104538006F20726573657429000D0A0A50726F67DF
:1045480072616D6D696E672D6572726F72212120BF
:10455800284374726C2B7220746F207265736574B3
:1045680029000D0A0A5465726D696E6174656420CC
:104578002D2072657374617274696E672E2E2E0019
:104588002100132A000D0A0A5352454320686F6C14
:1045980065212120284374726C2B7220746F20725D
:1045A80065736574290010034D00790020005000E0
:1045B80072006F0064000300000055534243090273
:1045C8002000010104803209040000020806500599
:1045D8000705010240000007058202400000008034
:1045E80000011F000000755461736B6572205553FC
:1045F80042204D5344204C6F616465722020312E57
:104608003030F8FFFF000A034D0061006E007500AE
:104618000A0343006F006E0066000A033000300092
:1046280030003100000000080001F800030002001B
:10463800080349006E007400001201100100000018
:10464800082504FC03000101020301006C46000078
:104658000E460000AE450000224600001846000045
:104668003846000004030904800000000000000A26
:1046780000000000000000000000656E61626C65CB
:104688002066696C6520726561642066726F6D20B2
:10469800746865204B696E65746973206465766912
:1046A8006365206279206472616767696E67207448
:1046B8006869732066696C6520746F20746865206A
:1046C8006469736B004D53444F53352E3000464197
:1046D8005431322020200055504C4F41445F44490A
:1046E800534B00555342204D53442052656164207A
:1046F800656E61626C65640A0D005553422052650F
:104708007365740A0D005553422053757370656EB6
:104718006465640A0D0055534220526573756D65D2
:104728000A0D00456E756D6572617465640D0A0049
:10473800534F46545741524542494E00010000121A
:104748000000000001577561000000009447000058
:1047580039420000000000000200010099470000F3
:10476800D105000045000200000000009D47000040
:10477800811500002500FFFF000004000000000074
:1047880000000000000000000000000057646F6790
:10479800006170700075736200008813C409E20438
:1047A800710239019C0068004E0027001A000D00B4
:1047B800070011278913C509E30472023901D100E2
:1047C8009D004F0035001B000E00000000A00640B1
:0C47D80000B0064000C0064001000000D8
:1047E40055534253000000000000000000018021E6
:0B47F400017001780906FCD57047FF3A
:0400000300000410E5
:00000001FF
